:06000000020064022BA1C6
:01000B0032C2
:0100130032BA
:03001B00022CA70D
:03002300022C3D6F
:03002B00022BB9EC
:03003300022BB8E5
:03003B00022B9005
:100064007581E8120C3C120C3C120C3C120C3C1234
:100074000C3C120C3C120C3C120C3C1200DDC20075
:1000840020010520083B80F8120623C20130040A2F
:10009400300507C204D200757C033000241209C164
:1000A4001209D9E57CB40103757C02300513C2053D
:1000B400757C00E57BB400030200C5200903120827
:1000C40014300306120C4E0200DA209109C2B53036
:1000D4000704C207D29902008475D703D20AC2AFBB
:1000E400C2D3C2D47400F8F9FAFBFCFDFEFFD2D3EC
:1000F400C2D47400F8F9FAFBFCFDFEFFC2D3D2D4DB
:100104007400F8F9FAFBFCFDFEFFD2D3D2D47400DC
:10011400F8F9FAFBFCFDFEFFC2D3C2D4120610129A
:1001240005A4D280D281D282D283D284D285D286CF
:10013400D287C2A0C2A1C2A2C2A3C2A4C2A5C2A69F
:10014400C2A7D290D291C2B5D2B0D2B1D2B2D2B3F8
:10015400C2B475F81FD2FDC29FD29ED29DD29CC25A
:100164009BC29AC299C298C2BED2BDC2BCC2BBC213
:10017400BAC2B9C2B8C2AFC2AED2ADD2ACC2ABC2BF
:10018400AAC2A9C2A875A901758933C28FC28EC239
:100194008DC28CC28BC28AC289C288758A00758C52
:1001A40000758B00758D00C2CFC2CEC2CDC2CCC249
:1001B400CBC2CAC2C9C2C8759E82759D2DC2DFC298
:1001C400DEC2DCC2DBC2DAC2D9C2D875D982758775
:1001D4000075CD3375CC3385CDCB85CCCA75EF6036
:1001E40075D800C289D2AFD2AE120C3C120C3C12AC
:1001F4000C3C120C3C120C3C120C3C1204BA1202C1
:100204005812091BC2B400D2B4120623C2B400D2DD
:10021400B4120623C2B400D2B4120623C2B400D26C
:10022400B4120623C20E75640078A47600120C3C46
:10023400120C3C120C3CC2AFC2AE120C46120C465D
:10024400120C46D2CAC28EC28CD2AFD2AEC208C27F
:1002540014C20A22757E00757F00E57FC20E754EBA
:1002640000D21175C60012268E121D8F75C6081293
:10027400268E121DA875C61012268E121DC175C6B3
:100284001A12268E121DDA200E03437E01C20E7549
:100294004E01C21175C60012268E121D8F75C60836
:1002A40012268E121DA875C61012268E121DC17537
:1002B400C61A12268E121DDA200E03437E02C20EC7
:1002C400754E02D21175C60112268E121D8F75C687
:1002D4000912268E121DA875C61112268E121DC172
:1002E40075C61A12268E121DDA200E03437E04C22E
:1002F4000E754E03C21175C60112268E121D8F751E
:10030400C60912268E121DA875C61112268E121D3C
:10031400C175C61A12268E121DDA200E03437E08FA
:10032400C20E754E04D21175C60212268E121D8F8E
:1003340075C60A12268E121DA875C61212268E12B2
:100344001DC175C61B12268E121DDA200E03437EB4
:1003540010C20E754E05C21175C60212268E121DEC
:100364008F75C60A12268E121DA875C61212268E05
:10037400121DC175C61B12268E121DDA200E0343F0
:100384007E20C20E754E06D21175C60312268E1239
:100394001D8F75C60B12268E121DA875C613122644
:1003A4008E121DC175C61B12268E121DDA200E0375
:1003B400437E40C20E754E07C21175C60312268EC7
:1003C400121D8F75C60B12268E121DA875C6131228
:1003D400268E121DC175C61B12268E121DDA200E22
:1003E40003437E80C20E754E08D21175C6041226D0
:1003F4008E121D8F75C60C12268E121DA875C6147A
:1004040012268E121DC175C61C12268E121DDA20EC
:100414000E05437F01E57FC20E754E09C21175C6F4
:100424000412268E121D8F75C60C12268E121DA85C
:1004340075C61412268E121DC175C61C12268E1284
:100444001DDA200E05437F02E57FC20E754E0AD2E7
:100454001175C60512268E121D8F75C60D12268EB5
:10046400121DA875C61512268E121DC175C61C1242
:10047400268E121DDA200E05437F04E57FC20E7519
:100484004E0BC21175C60512268E121D8F75C60D30
:1004940012268E121DA875C61512268E121DC17540
:1004A400C61C12268E121DDA200E03437F08E57F38
:1004B400C20E7564002275C61812268E8571768563
:1004C400727885737985747B75C61912268E857149
:1004D4007D857275E573B40005C2170204E4D21772
:1004E400E574B4460302059C7800757109757200C1
:1004F40075730975740088C612269E08E8B408EA64
:1005040075710175720075730175740088C61226C1
:100514009E08E8B410EA7571257572007573257527
:10052400740088C612269E08E8B418EA75C61A75BF
:10053400710075720075730075740012269E75C67D
:100544001B75710075720075730075740012269E18
:1005540075C61C7571007572007573007574001290
:10056400269E75763C757801757932757B00757DAC
:1005740000757514857671857872857973857B74B9
:1005840075C61812269E857D718575727573007502
:10059400744675C61912269EE579B40002D2062265
:1005A400D201D200D202C203C204C205C206C207EB
:1005B400C208D209C20CC20DC20EC20FC210C211AF
:1005C400C212C215D216C218D2191205FC756300E4
:1005D400D20275565875575812061078A4760075CD
:1005E400763C757801757932757700756400857984
:1005F4007A757C00757D002278247924760008D9E8
:10060400FB227824792476FF08D9FB2275500275E1
:10061400520275510575530A75543C75553C22D2E6
:100624000C754800754900754A4BE57E5401B401C8
:1006340021754E0012223B854CF0E52625F0F52667
:10064400854BF0E52535F0F52575F000E52435F00A
:10065400F524E57E5402B40224754E0112223B2097
:100664000A1B854CF0E52925F0F529854BF0E52892
:1006740035F0F52875F000E52735F0F527E57E54CB
:1006840004B40421754E0212223B854CF0E52C255E
:10069400F0F52C854BF0E52B35F0F52B75F000E5E6
:1006A4002A35F0F52AE57E5408B40821754E031264
:1006B400223B854CF0E52F25F0F52F854BF0E52EF8
:1006C40035F0F52E75F000E52D35F0F52DE57E5469
:1006D40010B41021754E0412223B854CF0E53225EE
:1006E400F0F532854BF0E53135F0F53175F000E584
:1006F4003035F0F530E57E5420B42021754E0512D6
:10070400223B854CF0E53525F0F535854BF0E53495
:1007140035F0F53475F000E53335F0F533E57E5406
:1007240040B44021754E0612223B854CF0E5382535
:10073400F0F538854BF0E53735F0F53775F000E521
:100744003635F0F536E57E5480B48021754E0712B7
:10075400223B854CF0E53B25F0F53B854BF0E53A33
:1007640035F0F53A75F000E53935F0F539E57F54A3
:1007740001B40121754E0812223B854CF0E53E255B
:10078400F0F53E854BF0E53D35F0F53D75F000E5BF
:100794003C35F0F53CE57F5402B40221754E091254
:1007A400223B854CF0E54125F0F541854BF0E540D1
:1007B40035F0F54075F000E53F35F0F53FE57F5441
:1007C40004B40421754E0A12223B854CF0E54425FD
:1007D400F0F544854BF0E54335F0F54375F000E55D
:1007E4004235F0F542E57F5408B40821754E0B12EA
:1007F400223B854CF0E54725F0F547854BF0E5466F
:1008040035F0F54675F000E54535F0F545C20C22A6
:10081400C209C201C200C20585767785797A757CE2
:1008240001C2AF120610D2AF1205FCD20422120983
:100834001BC2AFC209C201C200C205E579B4000BF4
:10084400757932757A32C20602085285797A757CD6
:10085400011206101205FCC2CA75CD3375CC33855E
:10086400CDCB85CCCAD2CAC2B400D2B4D204D2AFE2
:1008740022754802754900754A00E57E5401B401A9
:1008840006754E0012223BE57E5402B40206754EF4
:100894000112223BE57E5404B40406754E02122272
:1008A4003BE57E5408B40806754E0312223BE57EF0
:1008B4005410B41006754E0412223BE57E5420B445
:1008C4002006754E0512223BE57E5440B440067561
:1008D4004E0612223BE57E5480B48006754E071204
:1008E400223BE57F5401B40106754E0812223BE514
:1008F4007F5402B40206754E0912223BE57F54046C
:10090400B40406754E0A12223BE57F5408B4080667
:10091400754E0B12223B22754801754900754A0039
:10092400E57E5401B40106754E0012223BE57E5467
:1009340002B40206754E0112223BE57E5404B4044F
:1009440006754E0212223BE57E5408B40806754E25
:100954000312223BE57E5410B41006754E04122295
:100964003BE57E5420B42006754E0512223BE57EFD
:100974005440B44006754E0612223BE57E5480B4C2
:100984008006754E0712223BE57F5401B4010675BB
:100994004E0812223BE57F5402B40206754E09123A
:1009A400223BE57F5404B40406754E0A12223BE54B
:1009B4007F5408B40806754E0B12223B22301700F0
:1009C400C200782479807A24E6F70809DAFA200448
:1009D400031205FC22120C31788079B67A2420188F
:1009E40003020BF77563007A0078A5E6B400057876
:1009F40080020A4AB401057883020A4AB4020578DF
:100A040086020A4AB403057889020A4AB4040578BE
:100A14008C020A4AB40505788F020A4AB40605789E
:100A240092020A4AB407057895020A4AB40805787E
:100A340098020A4AB40905789B020A4AB40A05785E
:100A44009E020A4A78A1866908866A08866B12297A
:100A5400C2201905E56FB40A0F756F00770D0905FB
:100A640063770A090563C219200403020B22C21A20
:100A7400E56554F0C4B40003020A87D21A2430F79F
:100A8400090563E565540FB40006201A03020A9CA5
:100A9400D21A2430F7090563E56654F0C4B400069D
:100AA400201A03020AB2D21A2430F7090563E56654
:100AB400540FB40006201A03020AC7D21A2430F7CE
:100AC400090563E56754F0C4B40006201A03020A5A
:100AD400DDD21A2430F7090563E567540FB4000624
:100AE400201A03020AF2D21A2430F7090563E568D2
:100AF40054F0C4B40006201A03020B08D21A24309E
:100B0400F7090563E567540F2430F7090563772C6B
:100B140005637558B6C202D299056F020C30C21A29
:100B24007746090563E56554F0C4B40006201A034A
:100B3400020B3FD21A2430F7090563E565540FB45C
:100B44000006201A03020B54D21A2430F709056355
:100B5400E56654F0C4B40006201A03020B6AD21AE4
:100B64002430F7090563E566540FB40006201A0320
:100B7400020B7FD21A2430F7090563E56754F0C4E9
:100B8400B40006201A03020B95D21A2430F7090583
:100B940063E567540FB40006201A03020BAAD21AA5
:100BA4002430F7090563E56854F0C4B40006201A3C
:100BB40003020BC0D21A2430F7090563E567540F0A
:100BC4002430F7090563C218D219770D0905637734
:100BD4000A0905637558B6C202D29975C618122659
:100BE4008E857379E579B40005D206020C30C2060D
:100BF400020C30E6F70809DAFA78E6E6F70978E74E
:100C0400E6F709A77709A77609A77809A77909A7B5
:100C14007B09A77D09A77C09A76409740DF70974EA
:100C24000AF77563307558B6C202D2992278E6760F
:100C340000087600020C3B227E69DEFE227E0ADE7C
:100C4400FE227DFA120C3CDDFB22C203C20DE559E3
:100C5400B45303020CB8B45206020D4A020D8EB40A
:100C64004306122041020D8EB44611E55AB44306E0
:100C7400120DE0020D8E122CC0020D8EB45006121D
:100C84002045020D8EB45508C216120DD1020D8EE8
:100C9400B4570912220F120DD1020D8EB458061248
:100CA400222E020D8EB45A06122CAC020D8E120D99
:100CB400AA020D8EE55AB44106121376020D8EB4C3
:100CC4004309122059120DD1020D8EB44406121597
:100CD400A2020D8EB446061215E9020D8EB4480622
:100CE4001216AC020D8EB44C06121762020D8EB4AD
:100CF4004D09122140120DD1020D8EB44F0912215B
:100D040094120DD1020D8EB452061221E0020D8E02
:100D1400B45309122087120DD1020D8EB454061259
:100D240020E5020D8EB4550612180A020D8EB45732
:100D340006121992020D8EB447061218B2020D8ED5
:100D4400120DAA020D8EE55AB44406120F8F020D3D
:100D54008EB44606120EA2020D8EB44806120FE798
:100D6400020D8EB44C06121120020D8EB4550612DB
:100D7400124B020D8EB457061219D7020D8EB447CA
:100D840006121A22020D8E120DAA7559FF755AFF0A
:100D9400755BFF755CFF755DFF755EFF755FFF75C5
:100DA40060FF7561FF2279B677327563017558B6B5
:100DB400C202D2992279B6773109A74B09A74C0907
:100DC400A74D7563047558B6C202D2992279B677D5
:100DD400307563017558B6C202D29922E55B94302E
:100DE400B4000778A57600020E59B4010778A576F9
:100DF40001020E59B4020778A57602020E59B40313
:100E04000778A57603020E59B4040778A576040280
:100E14000E59B4050778A57605020E59B40607786D
:100E2400A57606020E59B4070778A57607020E596F
:100E3400B4080778A57608020E59B4090778A57690
:100E440009020E59B4110778A5760A020E59B41294
:100E54004178A5760BE55CC39430540FC4F577E56F
:100E64005DC39430540F3577F5777565007566006A
:100E7400756700756800E57754F0C4F567E5775445
:100E84000FF56878777C021227A6D218120832026E
:100E94000E9E120DAAC218020EA1120DD12275C601
:100EA40000120F1B75C601120F1B75C602120F1B11
:100EB40075C603120F1B75C604120F1B75C60512E7
:100EC4000F1B75C608120F1B75C609120F1B75C6BA
:100ED4000A120F1B75C60B120F1B75C60C120F1BC3
:100EE40075C60D120F1B75C610120F1B75C6111295
:100EF4000F1B75C612120F1B75C613120F1B75C676
:100F040014120F1B75C615120F1B75C618120F711C
:100F140075C619120F712212268E79B6E57154F036
:100F2400C42430F709E571540F2430F709E57254ED
:100F3400F0C42430F709E572540F2430F709E5733F
:100F440054F0C42430F709E573540F2430F709E54D
:100F54007454F0C42430F709E574540F2430F77541
:100F640063087558B6C202D2993002FD2212268E49
:100F740079B6A77109A77209A77309A774756304E1
:100F84007558B6C202D2993002FD22121F4C300DA0
:100F940003020FA9C20E75481A754900754A00125A
:100FA400223B300E06120DAA020FE679B6775209DB
:100FB400774409775409E55CF709E54C540F24306C
:100FC400F709E54DC4540F2430F709E54D540F24B7
:100FD40030F709770D09770A7563097558B6C202A7
:100FE400D29922E55BB4410BE55CB4430F121BA517
:100FF400020D8EB45206121C16020D8ED21478A461
:1010040076007564001223F2300D030210E91226F3
:101014008E30110985716D85726E02102785736D8E
:1010240085746EE56D54F0C4F565E56D540FF56691
:10103400E56E54F0C4F567E56E540FF568786E7C80
:10104400021227A6C20E754808754900754A001297
:10105400223B300E030210E9121FBE79B6200F0B9B
:10106400774809775609A75B021077774F097754B9
:1010740009A75B856D69856E6A122922E56B54F0B8
:10108400C4243079B9F709E56B540F2430F709E526
:101094006C54F0C42430F709E56C540F2430F7097C
:1010A400854C6D854D6E856D69856E6A122922E5C4
:1010B4006B54F0C4243079BDF709E56B540F243028
:1010C400F709E56C54F0C42430F709E56C540F2497
:1010D40030F709770D09770A75630D7558B6C202A2
:1010E400D29902111DD20D79B6774809775609A70E
:1010F4005B0977390977390977390977390977200D
:1011040009772009772009772009770D09770A756F
:10111400630D7558B6C202D299C21422E55BB4437A
:1011240006121C87020D8ED21478A4760075640012
:1011340012249F300D0302121412268E30110985D9
:10114400716D85726E02115285736D85746EE56DD5
:1011540054F0C4F565E56D540FF566E56E54F0C4BE
:10116400F567E56E540FF568786E7C021227A6C207
:101174000E754809754900754A0012223B300E036A
:10118400021214121FBE79B6200F0B774C09774454
:1011940009A75B0211A2774F09775409A75B856DF4
:1011A40069856E6A122922E56B54F0C4243079B93A
:1011B400F709E56B540F2430F709E56C54F0C424A7
:1011C40030F709E56C540F2430F709854C6D854DD3
:1011D4006E856D69856E6A122922E56B54F0C4240C
:1011E4003079BDF709E56B540F2430F709E56C54E9
:1011F400F0C42430F709E56C540F2430F709770D57
:1012040009770A75630D7558B6C202D2990212485D
:10121400D20D79B6774C09774409A75B0977390968
:1012240077390977390977390977200977200977D8
:101234002009772009770D09770A75630D7558B66B
:10124400C202D299C21422E55BB44306121CF8020E
:101254000D8ED21478A4760075640012254C300DDE
:101264000302133F12268E30110985716D85726E4B
:1012740002127D85736D85746EE56D54F0C4F56559
:10128400E56D540FF566E56E54F0C4F567E56E54EC
:101294000FF568786E7C021227A6C20E75480A758F
:1012A4004900754A0012223B300E0302133F121FFD
:1012B400BE79B6200F0B775509774409A75B021254
:1012C400CD774F09775409A75B856D69856E6A12DE
:1012D4002922E56B54F0C4243079B9F709E56B543D
:1012E4000F2430F709E56C54F0C42430F709E56C99
:1012F400540F2430F709854C6D854D6E856D6985D5
:101304006E6A122922E56B54F0C4243079BDF709C2
:10131400E56B540F2430F709E56C54F0C42430F71E
:1013240009E56C540F2430F709770D09770A7563C2
:101334000D7558B6C202D299021373D20D79B677DD
:101344005509774409A75B0977390977390977394A
:101354000977390977200977200977200977200947
:10136400770D09770A75630D7558B6C202D299C212
:101374001422E55BB4480CD21578A4760075640099
:1013840002138A021429E57E5401B40106755B3008
:101394001216ACE57E5402B40206755B311216AC2B
:1013A400E57E5404B40406755B321216ACE57E5433
:1013B40008B40806755B331216ACE57E5410B410FD
:1013C40006755B341216ACE57E5420B42006755BBA
:1013D400351216ACE57E5440B44006755B361216E1
:1013E400ACE57E5480B48006755B371216ACE57F9D
:1013F4005401B40106755B381216ACE57F5402B48F
:101404000206755B391216ACE57F5404B404067504
:101414005B411216ACE57F5408B40806755B4212B2
:1014240016AC021590B44C0CD21578A476007564F1
:101434000002143B0214DAE57E5401B40106755B24
:1014440030121762E57E5402B40206755B3112173E
:1014540062E57E5404B40406755B32121762E57EBD
:101464005408B40806755B33121762E57E5410B451
:101474001006755B34121762E57E5420B42006759D
:101484005B35121762E57E5440B44006755B361234
:101494001762E57E5480B48006755B37121762E5E7
:1014A4007F5401B40106755B38121762E57F54025C
:1014B400B40206755B39121762E57F5404B404065E
:1014C400755B41121762E57F5408B40806755B42E8
:1014D400121762021590B4550CD21578A4760075D3
:1014E40064000214EC021588E57E5401B40106750B
:1014F4005B3012180AE57E5402B40206755B3112A1
:10150400180AE57E5404B40406755B3212180AE521
:101514007E5408B40806755B3312180AE57E54102D
:10152400B41006755B3412180AE57E5420B4200604
:10153400755B3512180AE57E5440B44006755B3677
:1015440012180AE57E5480B48006755B3712180AB7
:10155400E57F5401B40106755B3812180AE57F541F
:1015640002B40206755B3912180AE57F5404B40408
:1015740006755B4112180AE57F5408B4080E755BC2
:101584004212180AD20D120DAA02159F300E031230
:101594000DB9300D03120DAA120DD1C21522E55B4F
:1015A400B45434D214121F4C300D030215DBE55D24
:1015B400C39430540F4549F549E55EC39430540F44
:1015C400C4F54AE55FC39430540F454AF54A75485B
:1015D4001912223B300E06120DAA0215E6120DD185
:1015E400C20EC21422C20E754E0075480B75490016
:1015F400754A0012223B754E0175480B75490075FA
:101604004A0012223B754E0275480B754900754A13
:101614000012223B754E0375480B754900754A004C
:1016240012223B754E0475480B754900754A001229
:10163400223B754E0575480B754900754A00122208
:101644003B754E0675480B754900754A0012223BDE
:10165400754E0775480B754900754A0012223B7593
:101664004E0875480B754900754A0012223B754EA9
:101674000975480B754900754A0012223B754E0ADC
:1016840075480B754900754A0012223B754E0B755F
:10169400480B754900754A0012223B200E06120DB4
:1016A400D10216AB120DAA22E55BB4410BE55CB482
:1016B400430F121A6D020D8EB45206121ABB020D9C
:1016C4008ED21420150F78A47600756400C20E30F3
:1016D4000E030217431223F2300D0302174CE55C8C
:1016E400C39430540FC4F549E55DC39430540F4599
:1016F40049F549E55EC39430540FC4F54AE55FC328
:101704009430540F454AF54AC3E54AF5F074009500
:10171400F0E549F5F0742095F0500302174C1226B9
:101724008E301109854971854A72021737854973CC
:10173400854A7412269E75480312223B300E1420EB
:101744001519120DB902175DD20D20150E120DAA2E
:1017540002175D201505120DD1C20EC21422E55BDD
:10176400B44306121B09020D8ED21420150F78A45F
:101774007600756400C20E300E030217EB12249F2C
:10178400300D030217F4E55CC39430540FC4F549DB
:10179400E55DC39430540F4549F549E55EC3943083
:1017A400540FC4F54AE55FC39430540F454AF54AD3
:1017B400C3E54AF5F0740095F0E549F5F074339506
:1017C400F050030217F412268E30110985497185F1
:1017D4004A720217DF854973854A7412269E75483A
:1017E4000412223B300E14201519120DB9021805EB
:1017F400D20D20150E120DAA021805201505120D82
:10180400D1C20EC21422E55BB44306121B57020D6B
:101814008ED21420150F78A47600756400C20E30A1
:101824000E0302189312254C300D0302189CE55C3C
:10183400C39430540FC4F549E55DC39430540F4547
:1018440049F549E55EC39430540FC4F54AE55FC3D6
:101854009430540F454AF54AC3E54AF5F0740095AF
:10186400F0E549F5F0743395F0500302189C122604
:101874008E301109854971854A720218878549732A
:10188400854A7412269E75480512223B300E142098
:101894001519120DB90218ADD20D20150E120DAA8C
:1018A4000218AD201505120DD1C20EC2142278A45F
:1018B4007600756400E55CB430030218CAB43103E1
:1018C4000218CA0219851225F912268EE55BB43076
:1018D40009E55C9430F57102195CB43109E55C9456
:1018E40030F57202195CB43209E55C9430F5730288
:1018F400195CB43309E55C9430F57402195CB434B2
:1019040009E55C9430F57102195CB43509E55C9421
:1019140030F57202195CB43609E55C9430F5730253
:10192400195CB43709E55C9430F57402195CB43879
:1019340009E55C9430F57102195CB43909E55C94ED
:1019440030F57202195CB44109E55C9430F5730218
:10195400195CE55C9430F57412269EC20E75480E2F
:10196400E55CC39430540FF549754A00121E6A3081
:101974000D0302198512223B300E03021985021948
:101984008E201509120DAA021991120DD12278A4E4
:101994007600756400E55CB430030219A4B4312602
:1019A400121E6A300D030219CAC20E75480CE55C9A
:1019B400C39430540FF549754A0012223B300E038C
:1019C4000219CA0219D3201509120DAA0219D61236
:1019D4000DD122121E6A300D030219F7C20E75488A
:1019E40010754900754A0012223B300E030219F7A4
:1019F400021A00201527120DAA021A2179B677526D
:101A040009775709E55BF709E54C2430F709770DA9
:101A140009770A7563067558B6C202D29922121E56
:101A24006A300D03021A42C20E75480F75490075DB
:101A34004A0012223B300E03021A42021A4B2015AE
:101A440027120DAA021A6C79B6775209774709E56D
:101A54005BF709E54C2430F709770D09770A7563BC
:101A6400067558B6C202D29922121EDB300D03024B
:101A74001AAE754811E55EB42B06754901021A8A3F
:101A8400B42D27754900E55FC39430540FC4F54A5B
:101A9400E560C39430540F854AF025F0F54A1222CC
:101AA4003B300E03021AAE021AB7201509120DAA12
:101AB400021ABA120DD122121EDB300D03021AFCD7
:101AC400754817E55EB42B06754901021AD8B42D82
:101AD40027754900E55FC39430540FC4F54AE560A7
:101AE400C39430540F854AF025F0F54A12223B3056
:101AF4000E03021AAE021B05201509120DAA021BC1
:101B040008120DD122121F4C300D03021B4A7548D6
:101B140012E55DB42B06754901021B26B42D277509
:101B24004900E55EC39430540FC4F54AE55FC3949D
:101B340030540F854AF025F0F54A12223B300E034B
:101B4400021B4A021B53201509120DAA021B56122E
:101B54000DD122121F4C300D03021B98754813E55A
:101B64005DB42B06754901021B74B42D2775490019
:101B7400E55EC39430540FC4F54AE55FC394305412
:101B84000F854AF025F0F54A12223B300E03021B62
:101B940098021BA1201509120DAA021BA4120DD133
:101BA40022121EDB300D03021BC37548147549FF56
:101BB400754AFF12223B300E03021BC3021BCC20CA
:101BC400154F120DAA021C1579B6E54DB400030297
:101BD4001BE7E54CB40106772B09021BE7B400DFD1
:101BE400772D09E54D54F0C42430F709772E09E523
:101BF4004D540F2430F709770D09770AE54DB400E9
:101C040006756305021C0E7563067558B6C202D2CA
:101C14009922121EDB300D03021C347548187549D5
:101C2400FF754AFF12223B300E03021C34021C3D96
:101C340020154F120DAA021C8679B6E54DB4000397
:101C4400021C58E54CB40106772B09021C58B40059
:101C5400DF772D09E54D54F0C42430F709772E09B8
:101C6400E54D540F2430F709770D09770AE54DB493
:101C74000006756305021C7F7563067558B6C202BB
:101C8400D29922121F4C300D03021CA575481575FC
:101C940049FF754AFF12223B300E03021CA5021CA9
:101CA400AE20154F120DAA021CF779B6E54DB4000B
:101CB40003021CC9E54CB40106772B09021CC9B404
:101CC40000DF772D09E54D54F0C42430F709772E51
:101CD40009E54D540F2430F709770D09770AE54DCE
:101CE400B40006756305021CF07563067558B6C228
:101CF40002D29922121F4C300D03021D167548168C
:101D04007549FF754AFF12223B300E03021D16026D
:101D14001D1F20154F120DAA021D6879B6E54DB49A
:101D24000003021D3AE54CB40106772B09021D3A63
:101D3400B400DF772D09E54D54F0C42430F709775A
:101D44002E09E54D540F2430F709770D09770AE57C
:101D54004DB40006756305021D617563067558B6BA
:101D6400C202D29922754801754900754A001222AF
:101D74003B120C3C120C3C22754802754900754A12
:101D84000012223B120C3C120C3C22754803301109
:101D94000985714985724A021DA485734985744A6F
:101DA40012223B2275480430110985714985724A13
:101DB400021DBD85734985744A12223B227548056C
:101DC40030110985714985724A021DD6857349858A
:101DD400744A12223B2275480EE54EB40006857102
:101DE40049021E45B40106857249021E45B4020625
:101DF400857349021E45B40306857449021E45B421
:101E04000406857149021E45B40506857249021E01
:101E140045B40606857349021E45B4070685744910
:101E2400021E45B40806857149021E45B40906859B
:101E34007249021E45B40A06857349021E4585741B
:101E440049754A0012223B22200A0878A4E604F6C7
:101E5400B4141078A47600756400E54EC44401F50A
:101E640064D20E222222E55BB43006754E00021EB7
:101E7400DAB43106754E01021EDAB43206754E022A
:101E8400021EDAB43306754E03021EDAB434067544
:101E94004E04021EDAB43506754E05021EDAB43657
:101EA40006754E06021EDAB43706754E07021EDAB0
:101EB400B43806754E08021EDAB43906754E0902A6
:101EC4001EDAB44106754E0A021EDAB44206754E95
:101ED4000B021EDAD20D22E55DB43006754E000207
:101EE4001F4BB43106754E01021F4BB43206754EBA
:101EF40002021F4BB43306754E03021F4BB4340663
:101F0400754E04021F4BB43506754E05021F4BB4C3
:101F14003606754E06021F4BB43706754E07021F70
:101F24004BB43806754E08021F4BB43906754E097A
:101F3400021F4BB44106754E0A021F4BB44206758C
:101F44004E0B021F4BD20D22E55CB43006754E00D9
:101F5400021FBCB43106754E01021FBCB4320675B3
:101F64004E02021FBCB43306754E03021FBCB434C8
:101F740006754E04021FBCB43506754E05021FBC1F
:101F8400B43606754E06021FBCB43706754E0702FA
:101F94001FBCB43806754E08021FBCB43906754E12
:101FA40009021FBCB44106754E0A021FBCB44206A6
:101FB400754E0B021FBCD20D2222856D6F856E708B
:101FC40079ADA76E19A76D197700197700197700F5
:101FD40079B0770A197700197700122721C378B5E9
:101FE400E6F5F0E56E95F0F56E18E6F5F0E56D951D
:101FF400F0F56DC3E54D856EF095F0E54C856DF01B
:1020040095F0403078B5E6256EF56E18E6356DF539
:102014006D78B5E6256EF56E18E6356DF56DE54D12
:10202400856EF0C395F0E54C856DF095F05005C2D2
:102034000F02203AD20F856F6D85706E221208143C
:1020440022300410C2AFC204D209D205757C0475D3
:102054007700D2AF227865760008E55BC39430F64A
:1020640008E55CC39430F608E55DC39430F608785F
:10207400757C011227A675C61912268E85757212F3
:10208400269E22C2AF78657600087600087600089E
:10209400E55BC39430F6787D7C011227A675C619DA
:1020A40012268E857D7112269EE57DB40109D20823
:1020B400C289D2A80220C1C2A8C289C208C201C270
:1020C40000C204D20575770085797AC2CA75CD330A
:1020D40075CC3385CDCB85CCCAD2CA120610D2AF0B
:1020E40022C2AF7865760008E55BC39430F608E554
:1020F4005CC39430F608E55DC39430F60878767CCA
:10210400011227A6E576B4000375763C75C618124D
:10211400268E85767112269EC201C200C204D205A3
:1021240075770085797AC2CA75CD3375CC3385CD80
:10213400CB85CCCAD2CA120610D2AF22C2AF786500
:10214400760008760008760008E55BC39430F678DC
:10215400787C011227A6C3E57894044003757801BE
:1021640075C61812268E85787212269EC201C20088
:10217400C204D20575770085797AC2CA75CD3375E4
:10218400CC3385CDCB85CCCAD2CA120610D2AF22AD
:10219400C2AF7865760008E55BC39430F608E55C69
:1021A400C39430F608E55DC39430F678797C011267
:1021B40027A6C3E57994C9400375793275C6181208
:1021C400268E85797312269EC20085797AE579B4C4
:1021D4000005D2060221DDC206D2AF227865760060
:1021E40008760008760008E55BC39430F6787B7CBB
:1021F400011227A6C3E57B94015003757B0075C6C5
:102204001812268E857B7412269E22E55AB4300855
:10221400C217755A00022221D217755A0175C619C0
:1022240012268E855A7312269E223006091205FC48
:102234001209C11209D922754B00754C00754D0065
:10224400200C271222F8C20B8548F7300BFD854F6E
:102254004BC20B8549F7300BFD854F4CC20B854AA9
:10226400F7300BFD854F4D1223751222F8120C3CEA
:10227400120C3CE548B41103022294B41203022266
:1022840094B41303022294B41703022294B41927BA
:10229400120C3C120C3C120C3C120C3C120C3C1266
:1022A4000C3C120C3C120C3C120C3C120C3C120C5C
:1022B4003C120C3C120C3CC20B75F700300BFD8534
:1022C4004F4BC20B75F700300BFD854F4CC20B759D
:1022D400F700300BFD854F4D122375200C15E54892
:1022E400B54B0DE549B54C08E54AB54D030222F757
:1022F400121E4C22E54EB40005C280022374B401C0
:1023040005C281022374B40205C282022374B40399
:1023140005C283022374B40405C284022374B40581
:1023240005C285022374B40605C286022374B40769
:1023340005C287022374B40805C2A0022374B40939
:1023440005C2A1022374B40A05C2A2022374B40B09
:1023540005C2A3022374B40C05C2A4022374B40DF1
:1023640005C2A5022374B40E05C2A6022374C2A733
:1023740022E54EB40005D2800223F1B40105D281D6
:102384000223F1B40205D2820223F1B40305D283FD
:102394000223F1B40405D2840223F1B40505D285E5
:1023A4000223F1B40605D2860223F1B40705D287CD
:1023B4000223F1B40805D2A00223F1B40905D2A185
:1023C4000223F1B40A05D2A20223F1B40B05D2A36D
:1023D4000223F1B40C05D2A40223F1B40D05D2A555
:1023E4000223F1B40E05D2A60223F1D2A722E55BA3
:1023F400B4300B754E0075C600D21102249EB43160
:102404000B754E0175C600C21102249EB4320B75C1
:102414004E0275C601D21102249EB4330B754E03CD
:1024240075C601C21102249EB4340B754E0475C6E0
:1024340002D21102249EB4350B754E0575C602C234
:102444001102249EB4360B754E0675C603D21102D2
:10245400249EB4370B754E0775C603C21102249E21
:10246400B4380B754E0875C604D21102249EB439D3
:102474000B754E0975C604C21102249EB4410B7536
:102484004E0A75C605D21102249EB4420B754E0B3A
:1024940075C605C21102249ED20D22E55BB4300B31
:1024A400754E0075C608D21102254BB4310B754E1A
:1024B4000175C608C21102254BB4320B754E027564
:1024C400C609D21102254BB4330B754E0375C609E8
:1024D400C21102254BB4340B754E0475C60AD211D1
:1024E40002254BB4350B754E0575C60AC21102257B
:1024F4004BB4360B754E0675C60BD21102254BB480
:10250400370B754E0775C60BC21102254BB4380B39
:10251400754E0875C60CD21102254BB4390B754E95
:102524000975C60CC21102254BB4410B754E0A75D0
:10253400C60DD21102254BB4420B754E0B75C60D58
:10254400C21102254BD20D22E55BB4300B754E004F
:1025540075C610D2110225F8B4310B754E0175C63B
:1025640010C2110225F8B4320B754E0275C611D291
:10257400110225F8B4330B754E0375C611C211024E
:1025840025F8B4340B754E0475C612D2110225F821
:10259400B4350B754E0575C612C2110225F8B43652
:1025A4000B754E0675C613D2110225F8B4370B7598
:1025B4004E0775C613C2110225F8B4380B754E08C0
:1025C40075C614D2110225F8B4390B754E0975C6B7
:1025D40014C2110225F8B4410B754E0A75C615D202
:1025E400110225F8B4420B754E0B75C615C21102C3
:1025F40025F8D20D22E55BB43009754E0075C61A74
:1026040002268DB43109754E0175C61A02268DB4A1
:102614003209754E0275C61A02268DB43309754EF9
:102624000375C61A02268DB43409754E0475C61B8B
:1026340002268DB43509754E0575C61B02268DB468
:102644003609754E0675C61B02268DB43709754EBC
:102654000775C61B02268DB43809754E0875C61C4D
:1026640002268DB43909754E0975C61C02268DB42F
:102674004109754E0A75C61C02268DB44209754E71
:102684000B75C61C02268DD20D2275B90185BC714D
:1026940085BD7285BE7385BF74228571BC8572BD8C
:1026A4008573BE8574BF75B90575B90275B904E53E
:1026B400B9B40005D2100226BFC2102278AE79AA9E
:1026C400E7F5F0E6A478B5F618E5F0F678AE79A962
:1026D400E7F5F0E6A4FA78B4E62AF6E5F034001853
:1026E400F678AE79A8E7F5F0E6A4FA78B3E62AF628
:1026F400E5F0340018F678AE79A7E7F5F0E6A4FA29
:1027040078B2E62AF6E5F0340018F678AE79A6E752
:10271400F5F0E6A478B1F5F0E625F0F6227828790C
:10272400B5770019770019770019770019770079C0
:10273400A87700197700197700C379ADE733F71943
:10274400E733F719E733F719E733F719E733F719DD
:10275400E733F719E733F719E733F7C379B0E7F548
:10276400F079A8E795F0FB79AFE7F5F079A7E7955D
:10277400F0FC79AEE7F5F079A6E795F0FD400A792B
:10278400A8EBF719ECF719EDF7B379B5E733F719B7
:10279400E733F719E733F719E733F719E733F7D8CE
:1027A40098228C0288058801770019DAFB796890F1
:1027B40027E21227CC9028321227CC9028821227A5
:1027C400CC9028D21227CC228D008C02E72323231D
:1027D4002407FBC3EB9336F61B18DAF81922000022
:1027E40000000000000000000000000000010000E4
:1027F40000000000000200000000000000030000D0
:1028040000000000000400000000000000050000BB
:1028140000000000000600000000000000070000A7
:102824000000000000080000000000000009000093
:10283400000000000000000000000000000A00008A
:10284400000000000014000000000000001E000052
:10285400000000000028000000000000003200001A
:1028640000000000003C00000000000000460000E2
:10287400000000000050000000000000005A0000AA
:1028840000000000000000000000000000640000E0
:102894000000000000C8000000000000012C00003F
:1028A40000000000019000000000000001F400009E
:1028B40000000000025800000000000002BC0000FC
:1028C400000000000320000000000000038400005A
:1028D40000000000000000000000000003E8000009
:1028E4000000000007D00000000000000BB800004A
:1028F400000000000FA0000000000000138800008A
:102904000000000017700000000000001B580000C9
:10291400000000001F400000000000002328C374D2
:10292400FF956A740F95695009756C99756B9902D6
:102934002971902972E56A540F93F56C902982E508
:102944006A54F0C42304FA93256CD4F56C1AEA9300
:102954003400D4F56B9029A2E569540F2304FA934B
:10296400256CD4F56C1AEA93356BD4F56B2200010F
:1029740002030405060708091011121314150000B8
:1029840000160032004800640080009601120128FD
:102994000144016001760192020802240240000011
:1029A4000256051207681024128015361792204823
:1029B4002304256028163072332835843840740087
:1029C400F568F567F566F565902A8CE56B540F9309
:1029D400F568902A9CE56BC4540F2304FA93256888
:1029E400D4F5681AEA933400D4F567902ABCE56AF2
:1029F400540F2304FA932568D4F5681AEA933567CB
:102A0400D4F567902ADCE56A54F0B40003022A2F57
:102A1400C4232314FA932568D4F5681AEA93356716
:102A2400D4F5671AEA933400D4F566902B18E56957
:102A3400540FB40003022A5B232314FA932568D4A9
:102A4400F5681AEA933567D4F5671AEA933566D4BC
:102A5400F5665003756501902B54E56954F0B40094
:102A640003022A8BC4232314FA932568D4F5681A25
:102A7400EA933567D4F5671AEA933566D4F5661A8E
:102A8400EA933565D4F565220001020304050607BF
:102A94000809101112131415000000160032004822
:102AA400006400800096011201280144016001764F
:102AB400019202080224024000000256051207682F
:102AC40010241280153617922048230425602816F6
:102AD40030723328358438400000409600008192DB
:102AE400000122880001638400020480000245760C
:102AF400000286720003276800036864000409600A
:102B040000045056000491520005324800057344F5
:102B140000061440000655360013107200196608AA
:102B2400002621440032768000393216004587524F
:102B34000052428800589824006553600072089639
:102B4400007864320085196800917504009830405B
:102B540001048576020971520314572804194304A9
:102B640005242880062914560734003208388608BC
:102B7400094371841048576011534336125829127F
:102B8400136314881468006415728640C0E0C0D0D2
:102B940020FEFD85F74FD0D0D0E0D20B32C0E0C08C
:102BA400D0300809D201C2B400D2B4D200C289D054
:102BB400D0D0E03232C0E0C0D0D55076755002207B
:102BC400080A201407D201C2B400D2B42006172088
:102BD4000814E57AB40003022BE59405F57AB400F1
:102BE40005D20085797AD5524975520230040AE536
:102BF40078B40005D57702D205D5533675530A301B
:102C0400040AE578B40105D57702D205D5542375B5
:102C1400543C30040AE578B40205D57702D205D5D0
:102C2400551075553C30040AE578B40305D5770290
:102C3400D205C2CFD0D0D0E032C0E0C0D0C000C0F6
:102C440001C2B5796330982CC298C0567462B556E7
:102C5400037556580556E557B55605D056022C76D9
:102C6400D0E0A856A699E6B40A0878567958E9F649
:102C7400D203000030991FC299B70005D202022C7A
:102C84009A209107D2B5D207022C9AC2B5A858E669
:102C9400F59908885817D001D000D0D0D0E0320080
:102CA40080FE320080FE322279B6E57EF709E57FA8
:102CB400F77563027558B6C202D2992279B6773392
:102CC40009773409773409773009773309774E095E
:102CD400773109773109770D09770A75630A7558D1
:062CE400B6C202D29922E3
:00000001FF
